:020000040000FA
:1000000000000000000000000000000000000000F0
:1000100000000000000000000000000000000000E0
:1000200000000000000000000000000000000000D0
:1000300000000000000000000000000000000000C0
:0200000400F00A
:08000000020000E40000020010
:080008000000040000000043A9
:08001000025704040000000087
:080018000000000000000000E0
:080020000000000000000000D8
:08002800000000000B000000C5
:080030000B0000000B000000B2
:08003800D00E0000D00E000004
:08004000D00E000000000000DA
:080048000000000000000000B0
:080050000000000000000000A8
:080058000000000000000000A0
:08006000000000000000000098
:080068002F0000002F00000032
:080070002F000000280300002E
:0800780028030000280300002A
:08008000000000000000000078
:0800880000000000010000006F
:08009000010000000100000066
:080098000AA001000AA001000A
:0800A0000AA0010000000001AC
:0800A80000000001000000014E
:0800B00000000003FFFFFFFF49
:0800B800FFFFFFFFFFFFFFFF48
:0800C000FFFFFFFFFFFFFFFF40
:0800C800FFFFFFFFFFFFFFFF38
:0800D000FFFFFFFFFFFFFFFF30
:0800D800FFFFFFFFFFFFFFFF28
:0800E000FFFF00000000010019
:0800E800000000000000000010
:0800F000000001000000000007
:0800F800000000BE4829695B0D
:020000040020DA
:08000000F0F1F9F2F0F0F0F16B
:020000040030CA
:0E0000000026040E000181000C800E800E0010
:00000001FF
